:020000040800F2
:100000000804002005010008290100082B01000850
:100010002D0100082F010008310100080000000038
:100020000000000000000000000000003301000894
:100030003501000800000000370100083901000800
:100040003B0100083B0100083B0100083B010008A0
:100050003B0100083B0100083B0100083B01000890
:100060003B0100083B0100083B0100083B01000880
:100070003B0100083B0100083B0100083B01000870
:100080003B0100083B0100083B0100083B01000860
:100090003B0100083B0100083B0100083B01000850
:1000A0003B0100083B0100083B0100083B01000840
:1000B0003B0100083B0100083B0100083B01000830
:1000C0003B0100083B0100083B0100083B01000820
:1000D0003B0100083B0100083B0100083B01000810
:1000E0003B0100083B0100083B010008DFF810D08D
:1000F00000F02EF8004800477D020008AFF30080B2
:10010000080400200D488047DFF83400016841F4FE
:10011000E0210160BFF34F8FDFF82800DFF82810DF
:1001200001600A4800477047FEE7FEE7FEE7FEE78A
:10013000FEE7FEE7FEE7FEE7FEE7FEE72701000831
:1001400024ED00E00CED00E00003FA05ED000008EE
:10015000064C074D06E0E06840F0010394E8070014
:1001600098471034AC42F6D3FFF7C4FF18030008D9
:100170003803000870B5194C8320206000256560A5
:10018000A56017486060012000F02EF86168084300
:10019000606014490D60086840F002000860206843
:1001A00040F48030206020688003FCD5206840F057
:1001B0008070206020688001FCD5606820F003001A
:1001C0006060606840F002006060606840F4800039
:1001D0006060086840F01000086070BD00100240C8
:1001E00000841D0000200240012804D0B0F5807F6B
:1001F00003DD012102E000202CE00021802801DD48
:10020000012200E000220A44402801DD012100E033
:1002100000210A44102801DD012100E000210A44E8
:10022000082801DD012100E000210A44042801DD45
:10023000012100E000210A44022801DD012100E043
:1002400000211144012801DD012000E000200844C4
:10025000C01D0001702800D10020704702E008C8CE
:10026000121F08C1002AFAD170477047002001E030
:1002700001C1121F002AFBD170470000C0B0FFF778
:1002800079FF00240AE02146084800F013F80849E5
:100290000860084600684DF82400641C402CF2DB1E
:1002A00000200349086000BFFEE700003803000893
:1002B000000000202DE9F04F4FF040024FF0000306
:1002C0004FF000044FF00005114FDFF848809342D3
:1002D00012D030F9139003FB01F606F03F0637F910
:1002E00016A009FB0AFB5C4438F916A009FB0AFBBF
:1002F0005D4403F10103EAE74FF000004FF0000115
:10030000C4FB0410C5FB0510BDE8F00F00BD0000E4
:10031000B803000838040008B804000800000020F2
:10032000040000005C020008BC0400080400002077
:10033000040400006C020008FF0FF60FD90FA80F8D
:10034000640F0E0FA70E2F0EA80D130D720CC50B08
:10035000100B530A9009C908000837077006AD054D
:10036000F0043B048E03ED025802D1015901F20062
:100370009C00580027000A0000000A0027005800CF
:100380009C00F2005901D1015802ED028E033B049A
:10039000F004AD05700637070008C9089009530A34
:1003A000100BC50B720C130DA80D2F0EA70E0E0F00
:1003B000640FA80FD90FF60FFF7F627F8A7D7D7AC9
:1003C0004276E3706E6AF262825A34511D47573C9E
:1003D000FC302825F9188C0C000074F307E7D8DAF4
:1003E00004CFA9C3E3B8CCAE7EA50E9D92951D8F18
:1003F000BE89838576829E8000809E8076828385FA
:10040000BE891D8F92950E9D7EA5CCAEE3B8A9C383
:1004100004CFD8DA07E774F300008C0CF91828250C
:10042000FC30573C1D473451825AF2626E6AE370C9
:1004300042767D7A8A7D627F00008C0CF91828252F
:10044000FC30573C1D473451825AF2626E6AE370A9
:1004500042767D7A8A7D627FFF7F627F8A7D7D7AA8
:100460004276E3706E6AF262825A34511D47573CFD
:10047000FC302825F9188C0C000074F307E7D8DA53
:1004800004CFA9C3E3B8CCAE7EA50E9D92951D8F77
:10049000BE89838576829E8000809E807682838559
:1004A000BE891D8F92950E9D7EA5CCAEE3B8A9C3E3
:0C04B00004CFD8DA07E774F30000000066
:04000005080000ED02
:00000001FF
